:0600000034C0FECFFDCF6D
:10000600FCCFFBCFFACFF9CFF8CFF7CFF6CFF5CFAE
:1000160055C0F3CFF2CFF1CFF0CFEFCFEECFEDCF8C
:100026001027E80364000A00010000100001100018
:1000360001000000000000000000000000007E0C2F
:10004600B69ECCDAFA0EFEDE00807E0CB69ECCDAC8
:10005600FA0EFEDE00800100020038000A000400ED
:100066003A000000F894EE27ECBBF1E0FBBFEBBFD3
:10007600E5BF8DE0A2E0BB27ED938A95E9F780E026
:1000860094E0A0E6ED930197E9F7ECE5F0E08591C1
:100096009591009761F0A591B59105901590BF01D6
:1000A600F00105900D920197E1F7FB01F0CFEFE526
:1000B600EDBFE4E0EEBFC0E6D1E035C0EA93FA93C7
:1000C600EFB7EA93BBD31BB10CB1E12FEC7189F406
:1000D600E52D5394F0E0E05AFE4F0083E8E0E51585
:1000E60009F455247394E8E0E71519F47724689425
:1000F60020F809911991E991EFBFF991E9911895C5
:100106001A937720F1F3E42D4394F0E0E05AFE4F82
:100116001081E8E0E41509F44424F8947A9478947C
:10012600E12F1991089568D298D2B9D1D60104D099
:10013600D501DBD0FACFFFCF95D2E4E4F0E081D34E
:1001460098D29AD2E0937001F09371019DD2E09318
:100156007201F0937301A1D2A4D2E0937401F093DB
:1001660075019BD25AD3E0937601F093770175D24D
:100176009ED2309711F4AA9A0BC09ED211F4A99A76
:1001860007C09ED211F4AC9A03C09ED209F4AB9A72
:10019600E0916C01F0916D018FD211F499D29CC05F
:1001A6008FD2D1F4ABE7B1E098D2E0917A01E0309A
:1001B60031F48ED298D214F0E1E09DD20CC0A09119
:1001C6007A01A13041F4AA9AA99AAC9AAB9A8BD239
:1001D60014F0E0E090D203C077D209F07DC024FE8F
:1001E60003C0EBE0F0E004C0E0917001F091710112
:1001F600E0937001F093710125FE3AC084D23097E6
:1002060099F426FC10C053D2309711F4AA980BC06B
:1002160053D211F4A99807C053D211F4AC9803C075
:1002260053D209F4AB980CC06ED23B9721F421D27D
:1002360023D2309709F002C0E89401C0689426F8EA
:1002460026FE10C034D2309711F4AA9A0BC034D2CD
:1002560011F4A99A07C034D211F4AC9A03C034D26F
:1002660009F4AB9A59D2139711F4E89426F80BC007
:100276001ED2A0E7B1E055D2EA0FFB1F0F0143D211
:10028600D001ED93FC9350D230F111D2309739F46E
:1002960024FC04C049D211F4AD9A01C0AD983CD2F9
:1002A600119731F447D2129711F4AD9A01C0AD9867
:1002B60033D2129731F43ED2149711F4AD9A01C09D
:1002C600AD982AD2139731F435D2189711F4AD9A16
:1002D60001C0AD9801C0AD9816D231D2E8D135D261
:1002E600E0937801F0937901D8C0BCD1E0E5F0E065
:1002F600A8D2BFD1C1D1E0937D01F0937E01C4D1D4
:10030600E0937F01F0938001C8D1CBD1E0938101C6
:10031600F0938201C2D181D2E0938301F0938401EC
:100326009CD118D2309711F4C19A0BC0C5D111F4E3
:10033600C09A07C0C5D111F4A89A03C0C5D109F463
:10034600C29AE0916801F0916901B6D111F407D221
:100356009CC0B6D1D1F4A8E8B1E0BFD1E091870145
:10036600E03031F4FCD100D214F0E1E005D20CC04B
:10037600A0918701A13041F4C19AC09AA89AC29A65
:10038600F3D114F0E0E0F8D103C09ED109F07DC0AE
:1003960022FE03C0EBE0F0E004C0E0917D01F091A5
:1003A6007E01E0937D01F0937E0123FE3AC0ECD1FD
:1003B600309799F427FC10C0CDD1309711F4C1982D
:1003C6000BC07AD111F4C09807C07AD111F4A8985D
:1003D60003C07AD109F4C2980CC0D6D13B9721F458
:1003E60048D14AD1309709F002C0E89401C0689418
:1003F60027F827FE10C0AED1309711F4C19A0BC072
:100406005BD111F4C09A07C05BD111F4A89A03C05E
:100416005BD109F4C29AC0D1139711F4E89427F876
:100426000BC098D1ADE7B1E07CD1EA0FFB1F0F01FD
:10043600ABD1D001ED93FC93B4D130F18BD1309791
:1004460039F422FC04C0ADD111F4AD9A01C0AD98C7
:10045600A3D1119731F4ABD1129711F4AD9A01C023
:10046600AD989AD1129731F4A2D1149711F4AD9A9E
:1004760001C0AD9891D1139731F499D1189711F421
:10048600AD9A01C0AD9801C0AD987ED158D162D168
:100496005CD1E0938501F09386012E96089577202E
:1004A60009F4A9C0E0919301F0E0E657FE4FFF93EF
:1004B600EF9326DEAF91BF91EC93E0919301EF5F4E
:1004C600E0939301A0919301A13021F4A0918A01B8
:1004D600A03F09F401C08CC0A0919301A93008F493
:1004E6008AC0A0919201AD3009F082C0E0918C01E2
:1004F600F0E0E6D0F1F560D1A13021F4E1E0F0E0E2
:100506005ED136C059D1A23061F45ED121F4E2E069
:10051600F0E055D105C0E0E0E0936801E0936901A1
:1005260027C04AD1A33021F5E3E0F0E048D150D10D
:100536005F014AD111F4689401C0E89422F8A091B1
:100546008E01A13011F4689401C0E89423F8A091BB
:100556009101A13040F0E0919101F0E0E0936A0151
:10056600F0936B0105C0E0E0E0936A01E0936B0154
:100576003FC0AAD0E9F520D1A13021F4E1E0F0E0B6
:1005860030D136C019D1A23061F41ED121F4E2E097
:10059600F0E027D105C0E0E0E0936C01E0936D0147
:1005A60027C00AD1A33021F5E3E0F0E01AD110D13B
:1005B6006F010AD111F4689401C0E89424F8A0915F
:1005C6008E01A13011F4689401C0E89425F8A09139
:1005D6009101A13040F0E0919101F0E0E0936E01CD
:1005E600F0936F0105C0E0E0E0936E01E0936F01C8
:1005F600E0E0E09393010895EFE2E7BBE0E0E8BBBB
:10060600EFE3E4BBE0E0E5BBEEEFE1BBE0E0E2BB3D
:10061600E3BFE2BFEFBDEEBDEDBDECBDE7BDE6BDA0
:10062600EBBDEABDE9BDE8BDE2BDE5BDE4BDE3BDA8
:10063600E9BFE5BFE2E0EBB9E0E9EAB9E6E8E0BD2B
:10064600E0E0E0BDE0E1E9B9E0E8E8B9E0E0E0BF1C
:10065600E6B9EDB9E6BF78940895E0E0E8BBE5BBFE
:10066600E2BB0895BA93AA932C978CE0A0E0B0E081
:100676000895AC85BD850895E8EEF3E0BBD0DF01B3
:10068600EAE0F0E0CAD00895F4DFE4E6F0E0B2D0A4
:10069600DF01EAE0F0E0C1D00895EBDFEAE0F0E048
:1006A6000895A8D0DF01EAE0F0E0B7D00895E09120
:1006B6007801F09179010895E130A0E0FA070895F4
:1006C600E230A0E0FA070895E330A0E0FA070895C3
:1006D600AA98A998AC98AB980895ED91FD9131969A
:1006E600FE93EE930895A0917B01B0917C01A83E04
:1006F600E3E0BE070895E0937A01E0E0E0937B0132
:10070600E0937C010895D3DFA0E7B1E0EE0FFF1F71
:10071600AE0FBF1F8FD00895A0917801B0917901D7
:100726000895EE0FFF1F0895A0916E01B0916F011D
:1007360011970895A0916E01B0916F010895DE01A1
:10074600AE0FBF1FEC91E2BB08953196A3E0B0E077
:1007560067D00895E0918501F09186010895C198CA
:10076600C098A898C2980895A0918801B09189016F
:10077600A83EE3E0BE070895E0938701E0E0E0933A
:100786008801E09389010895E5DFADE7B1E0C9DFAF
:10079600AE0FBF1F4FD00895A0918501B09186017D
:1007A6000895A0916A01B0916B0111970895A091E7
:1007B6006A01B0916B010895A0918B010895E093B1
:1007C6006801F09369010895A0918D01A130089503
:1007D600B0918F01A0E0E0919001F0E0EA2BFB2BB5
:1007E6000895E0936C01F0936D010895F195E195FC
:1007F600F04008950024112490E1AA0FBB1F001CAD
:10080600111C0E1A1F0A18F40E0E1F1E01C0A1603D
:100816009A9599F7FD01D0010895ECDFFD01089541
:10082600E894F7FF02C0E2DF6894EA23FB230EF4A4
:10083600DDDF0895ED91FC91119708951A930A93BF
:100846000895AC0FBD1F05900D928A95E1F70895A6
:00000001FF
